:100000000C94CB000C948A0B0C94B10B0C94E50768
:100010000C94E5070C94E5070C94F3000C94F300A2
:100020000C94F3000C94F3000C94F3000C94F30084
:100030000C94F3000C94F3000C94F3000C94F30074
:100040000C94D80B0C94F3000C94910E0C94C30EEA
:100050000C94F3000C94F3000C94F3000C94F30054
:100060000C94F3000C94F30020205375727665799C
:100070003D0020205374617475733D00202023538C
:100080006174733D002020414D534C3D0024524586
:10009000504F52542031202D312035002450524FE2
:1000A00043454544005374617274696E672047503C
:1000B0005320656E67696E6500475053206E6F74FC
:1000C00020726573706F6E64696E67005375727627
:1000D000657920526571756573742053656E74007F
:1000E0002453555256455920310024474554504F0A
:1000F0005300245245504F52542031202D31203589
:10010000002450524F4345454400436F6E74726F54
:100110006C6C6572205374617274696E672020394B
:10012000002A2A2050726F6772616D2053746172C9
:1001300074202A2A000000000800020100000304C5
:100140000700000000000000000102040810204029
:100150008001020408102001020408102004040495
:100160000404040404020202020202030303030360
:1001700003000000002300260029000000000025E5
:100180000028002B0000000000240027002A0000A7
:100190008602F30EE10211241FBECFEFD8E0DEBFCE
:1001A000CDBF11E0A0E0B1E0E6E7FAE202C00590C1
:1001B0000D92A83BB107D9F723E0A8EBB1E001C04D
:1001C0001D92A43BB207E1F711E0C4E9D1E004C0FD
:1001D0002297FE010E945B12C039D107C9F70E9425
:1001E000B6110C942E150C94000081E090E09093D1
:1001F000300280932F020895CF93DF93EC016EE0DD
:1002000071E083E193E00E94A50FCA30D1052CF480
:1002100060E383E193E00E94A70F4AE050E0BE0153
:1002200083E193E0DF91CF910C9467104F925F923E
:100230006F927F928F929F92AF92BF92CF92DF92F6
:10024000EF92FF920F931F93CF93DF93CDB7DEB75B
:100250002C970FB6F894DEBF0FBECDBF809167021A
:10026000909168020E946E146B017C018BE6D81A93
:1002700085E4E80A85EFF80AC0925502D09256024A
:10028000E0925702F09258028091690290916A02BE
:100290000E946E144B015C01E0E88E1AE5EB9E0AA9
:1002A000E2EAAE0AEAEFBE0A8092590290925A023E
:1002B000A0925B02B0925C028E010F5F1F4F88E03C
:1002C000F80111928A95E9F7C701B60120E03DE2F5
:1002D00041E351E00E940C122B013C012F5B29836A
:1002E000C501B40120E836E948E950E00E940C124B
:1002F00069877A878B879C872F5B2A83C301B2012A
:1003000020E834E84EE150E00E940C12205D2B837F
:1003100080E4482E82E4582E8FE0682E712C698587
:100320007A858B859C85A30192010E940C12205D29
:100330002C83C701B60120E834E84EE150E00E946A
:100340000C1225E835E441E050E00E940C122F59D0
:100350002D83C501B401A30192010E940C1222EC6D
:1003600032EA40E050E00E940C122F592E836AEAD4
:1003700071E089E292E00E945E117E01F7E0EF0EEB
:10038000F11CF80161918F0189E292E00E94A211B3
:100390000E151F05B1F72C960FB6F894DEBF0FBEF1
:1003A000CDBFDF91CF911F910F91FF90EF90DF9024
:1003B000CF90BF90AF909F908F907F906F905F9005
:1003C0004F9008958F929F92AF92BF92CF92DF92FB
:1003D000EF92FF924B015C010E94220C6B017C01A9
:1003E000C80CD91CEA1CFB1C0E94220CC616D7069E
:1003F000E806F906C8F7FF90EF90DF90CF90BF9026
:10040000AF909F908F900895CF93DF9362E083E049
:100410000E94DD0C26E040E855E260E070E083E1F8
:1004200093E00E942F0E64EF71E080E090E00E9464
:10043000510C40E855E260E070E08CEB91E00E94E6
:10044000E80864EF71E080E090E00E94510C61E206
:1004500071E083E193E00E94B20F42E050E065EF6B
:1004600070E081E00E946A0B6AE071E083E193E052
:100470000E94740FC8E0D0E060E171E083E193E096
:100480000E94A50F4AE050E0BE0183E193E00E9484
:10049000671068EE73E080E090E00E94E20121972F
:1004A00059F783E193E00E94AE0F61E071E08CEBBD
:1004B00091E00E94B20F64EC79E080E090E00E944D
:1004C000E20162EF70E08CEB91E0DF91CF910C9450
:1004D000B20F65EA70E083E193E00E94B20F6CE92D
:1004E00070E08CEB91E00E94B20F6CEA7DE080E05E
:1004F00090E00E94E2016DE870E08CEB91E00E94D8
:10050000B20FE091BA01F091BB0109946AEA71E07F
:1005100089E292E00E94481168E771E08BED91E07A
:100520000E94481162E171E081EE91E00E94481161
:1005300066E171E087EE91E00E9448116AE171E0A6
:100540008DEE91E00E9448116EE171E083EF91E041
:100550000E94481162E271E089EF91E00E94481127
:1005600066E271E08FEF91E00E9448116AE271E06B
:1005700085E092E00E9448116EE271E08BE092E02B
:100580000E94481162E371E081E192E00E9448110B
:1005900066E371E087E192E00E9448116AE371E04E
:1005A0008DE192E00E9448116EE371E083E292E0F7
:1005B0000E94481120E049E068E08CEB91E00C9447
:1005C000B808CF93DF938CEB91E00E945F08C9E2FB
:1005D000D2E02697CE010E94DA1081E0CB3DD80709
:1005E000C1F789E292E0DF91CF910C94DA104F923B
:1005F0005F926F927F928F929F92AF92BF92CF92B3
:10060000DF92EF92FF92CF93DF93109270021092DD
:100610006F021092A8028AEA91E0909342028093BE
:10062000410282E3E6E7F2E0DF011D928A95E9F7F5
:10063000109275022091A802243259F14CED55E038
:1006400060E070E08CEB91E00E94B11041E050E07E
:1006500068EA72E08CEB91E00E94B710909372020E
:1006600080937102181619067CF069EB70E083E143
:1006700093E00E94B20F81E090E090936602809335
:10068000650289E090E01DC28091A8028093750206
:10069000D1CF81E090E09093740280937302209315
:1006A00076028CEB91E00E948E0718161906A4F4CE
:1006B0008CEB91E00E9400078093750220917302F9
:1006C00030917402F901EA58FD4F80832F5F3F4F4C
:1006D0003093740220937302809175028A3009F777
:1006E000E0917302F0917402EB58FD4F108268E7BD
:1006F00071E086E792E00E9495147C01909342029B
:100700008093410262E471E00E94A314892B29F4D2
:100710000E94690281E090E0D4C16AE471E0C701FF
:100720000E94A314892B09F04FC068E771E080E0B4
:1007300090E00E94951490936C0280936B020E944B
:100740006E1460933D0270933E0280933F0290933B
:10075000400268E771E080E090E00E949514909379
:100760006C0280936B020E94501480933C0268E7F5
:1007700071E080E090E00E94951490936C02809369
:100780006B020E94501480933B0260913D02709175
:100790003E0280913F02909140026058724C8A4222
:1007A0009D4E20913C02621B710981099109609361
:1007B0003D0270933E0280933F02909340020E945C
:1007C0007B0A82E090E07DC161E571E0C7010E9493
:1007D000A314892B09F04BC068E771E080E090E03A
:1007E0000E94951490936C0280936B020E945014A7
:1007F00080933A0268E771E080E090E00E949514EF
:1008000090936C0280936B0268E771E080E090E067
:100810000E94951490936C0280936B020E94501476
:100820008093390268E771E080E090E00E949514BF
:1008300090936C0280936B0268E771E080E090E037
:100840000E94951490936C0280936B0268E771E0AC
:1008500080E090E00E94951490936C0280936B026C
:100860000E9450148093370283E090E02AC169E52A
:1008700071E0C7010E94A314892BF1F468E771E0CD
:1008800080E090E00E94951490936C0280936B023C
:100890000E945014909334028093330268E771E011
:1008A00080E090E00E94951490936C0280936B021C
:1008B0000E9450148093380264E671E080914102F6
:1008C000909142020E94A314892BC1F568E771E060
:1008D00080E090E00E94951490936C0280936B02EC
:1008E00068E771E080E090E00E94951490936C02BC
:1008F00080936B0268E771E080E090E00E949514BD
:1009000090936C0280936B0268E771E080E090E066
:100910000E94951490936C0280936B0268E771E0DB
:1009200080E090E00E94951490936C0280936B029B
:100930000E94501490933202809331026CE671E071
:1009400080914102909142020E94A314892B09F0E8
:10095000B6C068E771E080E090E00E949514909343
:100960006A028093690268E771E080E090E00E948B
:100970009514909368028093670268E771E080E0C5
:1009800090E00E94951490934602809345020E9445
:10099000501490934402809343020E941601E09108
:1009A0006902F0916A02808180934B028D3249F492
:1009B00083E5809349023196F0936A02E0936902DD
:1009C00003C08EE480934902E0916702F0916802CF
:1009D000808180934B028D3249F487E580934702F2
:1009E0003196F0936802E093670203C085E4809338
:1009F0004702C0906902D0906A02C6010E946E143C
:100A000020E4822E22E4922E2FE0A22EB12CA5010A
:100A100094010E940C1229013A0120936102309343
:100A200062024093630250936402C0916702D091C6
:100A30006802CE010E946E14A50194010E940C125E
:100A400049015A0120935D0230935E0240935F0298
:100A500050936002C6010E946E146B017C01A301D9
:100A6000920160E472E48FE090E00E94C611C61A21
:100A7000D70AE80AF90AC0925102D0925202E092D3
:100A80005302F0925402CE010E946E146B017C015D
:100A9000A501940160E472E48FE090E00E94C61129
:100AA000C61AD70AE80AF90AC0924D02D0924E023D
:100AB000E0924F02F092500284E090E002C080E0A9
:100AC00090E0DF91CF91FF90EF90DF90CF90BF90BB
:100AD000AF909F908F907F906F905F904F90089510
:100AE0000E945D0B26E0289FB001299F700D112404
:100AF00065527E4F83E193E00E94970F68E771E0B3
:100B000083E193E00E94A50F0E94550B4AE050E05C
:100B1000BC0183E193E00E94671064E771E083E128
:100B200093E00E94A50F0E94650B4AE050E0BC01D3
:100B300083E193E00E94671068E771E083E193E04E
:100B40000E94A50F0E943D0B4AE050E0BC0183E1EA
:100B500093E00E9467100E94450B0E94FC000E94D7
:100B60004D0B0E94FC0067E771E083E193E00E9477
:100B7000A50F69E272E083E193E00E94970F67E7B7
:100B800071E083E193E00E94A50F409161025091D2
:100B9000620260916302709164022AE030E083E1B6
:100BA00093E00E946F106AE771E083E193E00E9496
:100BB000A50F4091510250915202609153027091E1
:100BC00054022AE030E083E193E00E941D1060911E
:100BD000490283E193E00E94A70F67E771E083E198
:100BE00093E00E94A50F40915D0250915E026091DA
:100BF0005F02709160022AE030E083E193E00E949E
:100C00006F106AE771E083E193E00E94A50F4091C5
:100C10004D0250914E0260914F02709150022AE0B5
:100C200030E083E193E00E941D106091470283E170
:100C300093E00E94A70F65E870E083E193E00E94D3
:100C4000740F60914302709144024AE050E083E1E6
:100C500093E00E9467106CE770E083E193E00E94EC
:100C6000740F4AE050E06091380283E193E00E9403
:100C70007C1062E770E083E193E00E94740F4AE029
:100C800050E06091370283E193E00E947C108091F4
:100C90003102909132021816190684F468E670E069
:100CA00083E193E00E94740F6091310270913202EF
:100CB0004AE050E083E193E00E94671083E193E013
:100CC0000E94AE0F83E193E00C94A80DCF93DF93C5
:100CD00010926602109265020E94F70290937002D1
:100CE00080936F02C0913502D09136020E944D0B65
:100CF000C817D90759F10E94650B8A3D974034F413
:100D000082E090E090936602809365020E947005F5
:100D10000E944D0B90933602809335020E944D0B3A
:100D200065E070E00E94D61190936E0280936D0290
:100D3000892B61F46AEE70E08CEB91E00E94B20FB7
:100D40000E94F7029093700280936F0280913802A4
:100D50008430E0F080912F02909130020197B1F43D
:100D600060EE70E08CEB91E00E94B20F6CEC70E0F2
:100D700083E193E00E94B20F64E670E080E090E0CF
:100D80000E94E2011092300210922F022091A802DC
:100D90008091730290917402833091051CF420E0DD
:100DA0000196FACF2093A802909374028093730265
:100DB00044EF51E060E070E083E193E00E94B11005
:100DC00042E050E068EA72E083E193E00E94B710ED
:100DD00090937202809371021816190674F4809130
:100DE000A802833751F48091A902813331F481E064
:100DF00090E09093300280932F02DF91CF9108957D
:100E00002091ED023091EE0228173907B9F4909144
:100E1000AB028091AC02981789F0E091AB02F0E050
:100E2000E355FD4F80812091AB0230E02F5F3F4FB3
:100E30002F7333272093AB0290E008958FEF9FEF3D
:100E400008951F93CF93DF93DC015C968D919C9165
:100E50005D97009749F481E090E013969C938E9300
:100E6000129780E090E03BC05196ED91FC91529733
:100E700050962C915097322F30951FB75E964C911B
:100E80005E9741FB772770F941FD6095F8944081AA
:100E9000772311F0422B01C043234083EC012197BB
:100EA000F1F748E0508160FF02C0522B01C053238C
:100EB0005083EC012197F1F76695415099F78081B5
:100EC000772311F0832301C0822B80831FBF5C96A0
:100ED0008D919C915D970197F1F781E090E0DF9112
:100EE000CF911F91089508952091ED023091EE0267
:100EF0002817390781F49091AB028091AC029817C2
:100F000051F0E091AB02F0E0E355FD4F808199276D
:100F100087FD909508958FEF9FEF08952091ED0242
:100F20003091EE022817390771F48091AC022091BC
:100F3000AB0290E0805C9F4F821B910960E470E0FF
:100F40000E94D611089580E090E00895E091ED02AE
:100F5000F091EE02E817F90769F4A389B4899C912E
:100F60008589809589238C931092EE021092ED0270
:100F700081E0089580E00895CF93DF93EC018A8D9E
:100F80009B8D892BF1F08091ED029091EE028C17F0
:100F90009D07B9F0009711F00E94A6078E8D8E7FF5
:100FA0008E8F1092AC021092AB02D093EE02C093DF
:100FB000ED02EB89FC8980819D89892B808381E00A
:100FC00001C080E0DF91CF9108951F920F920FB67C
:100FD0000F9211242F933F934F935F936F937F93BF
:100FE0008F939F93AF93BF93EF93FF93E091ED02A5
:100FF000F091EE02309709F451C0868DA685B78531
:10100000958581FF04C08C91892329F447C08C9178
:10101000892309F043C0A389B4899C91858980956F
:1010200089238C93868997890197F1F7208D318DDB
:10103000A685B785758558E040E0C9010197F1F7AD
:10104000842F90E095958795482F6C91672309F040
:101050004068515091F7868D81FD40958091AC029A
:1010600090E001968F7399272091AB02281749F0E1
:10107000A091AC02B0E0A355BD4F4C938093AC025D
:1010800003C0868D8160868F828D938D0197F1F7E5
:10109000A389B4898C919589892B8C93FF91EF91C9
:1010A000BF91AF919F918F917F916F915F914F9180
:1010B0003F912F910F900FBE0F901F90189520E831
:1010C00031E0FC01318320830C94A6071F93CF935A
:1010D000DF93EC01162F6E8D6695617081E06827B5
:1010E000812F0E94160D61E0812F0E94DD0C812F5F
:1010F00090E0FC01E75BFE4FE491E88BFC01E35AD2
:10110000FE4FE491F0E0EE0FFF1FE558FE4F859192
:1011100094919A8B898BDF91CF911F9108951F93A2
:10112000CF93DF93EC01162F60E0812F0E94DD0C3E
:101130008E8D81FD04C061E0812F0E94160D1C87F9
:10114000812F90E0FC01E75BFE4FE491ED87FC010D
:10115000E35AFE4FE491F0E0EE0FFF1FEF58FE4F11
:10116000859194919F878E87DF91CF911F910895EC
:10117000FF920F931F93CF93DF93EC01F62E522F24
:101180001B821A8208EE13E020E030E00C831D83FE
:101190002E833F8380E891E0998388831F8A1E8A8B
:1011A000198E188E1B8E1A8E1D8E1C8E8E8D8E7F24
:1011B00050FB81F98E8F642FCE010E9466086F2D3F
:1011C000CE01DF91CF911F910F91FF900C948F086A
:1011D000CF93DF93EC019A01AB011B8E1A8E198E0F
:1011E000188E1F8A1E8A60E079E08DE390E00E94ED
:1011F0000C12C9012430310520F0B9016350710986
:1012000002C061E070E07D8F6C8FEC85E63108F004
:1012100068C0B901769567956431710518F063511E
:10122000710902C061E070E07F8B6E8B069718F049
:10123000C901059702C081E090E0998F888FC901AC
:10124000880F991F820F931F96958795969587957E
:101250008D30910510F00C9702C081E090E09B8FDB
:101260008A8F20916800E83050F091E0EE3008F469
:1012700090E081E001C0880F9A95EAF701C084E010
:10128000822B809368002C85283038F02E3040F077
:10129000263148F48CE690E008C08DE690E005C069
:1012A0008BE690E002C080E090E09C8B8B8B283036
:1012B00030F481E001C0880F2A95EAF70DC0822F33
:1012C00090E02E3010F4089701C00E9791E001C015
:1012D000990F8A95EAF7892F8D8B8C8D9D8D0197BB
:1012E000F1F7CE01DF91CF910C94BC076F927F9202
:1012F0008F929F92AF92BF92CF92DF92EF92FF9226
:101300000F931F93CF93DF93EA012CE3C22ED12CCE
:10131000E12CF12CA70196010E94EA116883CA0111
:10132000B901A70196010E94EA116983CA01B901B6
:1013300028E130E040E050E00E94EA1149015A0102
:101340006A83CA01B9016C5F7F4F8F4F9F4F27E0BF
:1013500030E040E050E00E94EA116F5F6B8300E0F4
:1013600010E0980140E054E6652E712C60E9C62E2D
:10137000DD24D394E42FF0E0EE54F84F7F0183E0B6
:10138000E822FF24E114F10489F4CF01B3010E94A3
:10139000D611892B29F08EE691E0A0E0B0E00AC0DA
:1013A000CF01B6010E94D611892BA9F38DE691E0F9
:1013B000A0E0B0E0080F191F2A1F3B1FD901C80188
:1013C000AA27BB2788169906AA06BB0610F04F5F0E
:1013D000D1CF4E83E114F10499F4CF0164E670E0BB
:1013E0000E94D611892B29F08EE691E0A0E0B0E0B2
:1013F0000BC0CF0160E971E00E94D611892BA1F3E7
:101400008DE691E0A0E0B0E0081B190B2A0B3B0B26
:10141000801A910AA20AB30ACF0164E670E00E9422
:10142000D6119C01CF0160E971E00E94D611ECE871
:10143000F1E0A0E0A13059F4E114F10451F42115D8
:10144000310511F04DE106C00097E1F302C0408183
:1014500001C04CE150E060E070E084169506A606FD
:10146000B70640F0841A950AA60AB70AAF5F31960C
:10147000AC3001F7AF5FAD8383948C82DF91CF9165
:101480001F910F91FF90EF90DF90CF90BF90AF90A2
:101490009F908F907F906F900895CF92DF92EF9200
:1014A000FF926B017C018091FF0290910003A0915B
:1014B0000103B0910203C816D906EA06FB0671F0D3
:1014C00043E053E0C701B6010E947609C092FF02D3
:1014D000D0920003E0920103F0920203FF90EF909C
:1014E000DF90CF9008950E944D0A8091090390E00B
:1014F0008E54984F08950F931F936093FB0270933F
:10150000FC028093FD029093FE020091060110916F
:1015100007012091080130910901060F171F281FAC
:10152000391F0093F3021093F4022093F5023093D5
:10153000F60282E090E09093F2028093F1020E9422
:10154000220C6093F7027093F8028093F902909353
:10155000FA021F910F910895CF92DF92EF92FF92BE
:101560000F931F930E94220CC090F702D090F802B4
:10157000E090F902F090FA026C197D098E099F093A
:101580000091FB021091FC022091FD023091FE02BD
:10159000683E734081059105D8F00F5F1F4F2F4FB4
:1015A0003F4F0093FB021093FC022093FD02309307
:1015B000FE0248EEC40E43E0D41EE11CF11CC092B2
:1015C000F702D092F802E092F902F092FA02CACF42
:1015D0008091F3029091F402A091F502B091F6028D
:1015E000081719072A073B07C8F1E091EF02F091AD
:1015F000F002309799F10995611571058105910502
:1016000019F00E947B0A2AC080910601909107017F
:10161000A0910801B09109014091FB025091FC0298
:101620006091FD027091FE02840F951FA61FB71FE7
:101630008093F3029093F402A093F502B093F60224
:1016400081E090E02091F1023091F202232B11F41D
:1016500080E090E09093F2028093F1026091FB02AF
:101660007091FC028091FD029091FE021F910F91FA
:10167000FF90EF90DF90CF9008950E94AC0A0E94F7
:101680004D0A8091050390E008950E94AC0A0E94E3
:101690004D0A8091040390E008950E94AC0A0E94D4
:1016A0004D0A8091030390E008950E94AC0A0E94C5
:1016B0004D0A8091070390E008950E94AC0A0E94B1
:1016C0004D0A8091080390E008950E94AC0A0C94A2
:1016D000730A08958230E8F4E82FF0E0EE0FFF1F60
:1016E000E65FFE4F71836083813041F08091690035
:1016F0008C7F842B80936900E89A0895809169001B
:10170000440F551F440F551F837F842B809369001E
:10171000E99A08951F920F920FB60F9211242F93FA
:101720003F934F935F936F937F938F939F93AF9369
:10173000BF93EF93FF93E0910A01F0910B0109959C
:10174000FF91EF91BF91AF919F918F917F916F9199
:101750005F914F913F912F910F900FBE0F901F906F
:1017600018951F920F920FB60F9211242F933F934B
:101770004F935F936F937F938F939F93AF93BF9399
:10178000EF93FF93E0910C01F0910D010995FF910A
:10179000EF91BF91AF919F918F917F916F915F91E9
:1017A0004F913F912F910F900FBE0F901F90189562
:1017B0001F920F920FB60F9211242F933F938F9386
:1017C0009F93AF93BF9380910B0390910C03A091D3
:1017D0000D03B0910E0330910A0323E0230F2D3740
:1017E00020F40196A11DB11D05C026E8230F029625
:1017F000A11DB11D20930A0380930B0390930C034A
:10180000A0930D03B0930E0380910F0390911003EA
:10181000A0911103B09112030196A11DB11D8093F7
:101820000F0390931003A0931103B0931203BF9181
:10183000AF919F918F913F912F910F900FBE0F907D
:101840001F9018952FB7F89460910B0370910C03BB
:1018500080910D0390910E032FBF08953FB7F89428
:1018600080910F0390911003A0911103B091120386
:1018700026B5A89B05C02F3F19F00196A11DB11DEB
:101880003FBF6627782F892F9A2F620F711D811D08
:10189000911D42E0660F771F881F991F4A95D1F767
:1018A0000895CF92DF92EF92FF92CF93DF936B0177
:1018B0007C010E942E0CEB01C114D104E104F1045F
:1018C00089F00E94C5110E942E0C6C1B7D0B683E96
:1018D000734090F381E0C81AD108E108F108C851BB
:1018E000DC4FEACFDF91CF91FF90EF90DF90CF9068
:1018F0000895789484B5826084BD84B5816084BD88
:1019000085B5826085BD85B5816085BDEEE6F0E078
:10191000808181608083E1E8F0E0108280818260D4
:101920008083808181608083E0E8F0E08081816055
:101930008083E1EBF0E0808184608083E0EBF0E085
:10194000808181608083EAE7F0E080818460808329
:1019500080818260808380818160808380818068D3
:1019600080831092C1000895833081F028F4813083
:1019700099F08230A1F008958730A9F08830B9F04D
:101980008430D1F4809180008F7D03C080918000ED
:101990008F7780938000089584B58F7702C084B5D7
:1019A0008F7D84BD08958091B0008F7703C08091B2
:1019B000B0008F7D8093B0000895CF93DF9390E0C7
:1019C000FC01E75BFE4F2491FC01E35AFE4F84913A
:1019D000882349F190E0880F991FFC01EB57FE4FD7
:1019E000A591B49185589E4FFC01C591D4919FB7A4
:1019F000611108C0F8948C91209582238C93888182
:101A000082230AC0623051F4F8948C91322F3095C1
:101A100083238C938881822B888304C0F8948C91D3
:101A2000822B8C939FBFDF91CF9108950F931F93CB
:101A3000CF93DF931F92CDB7DEB7282F30E0F901A7
:101A4000EB5CFE4F8491F901E75BFE4F1491F901C5
:101A5000E35AFE4F04910023C9F0882321F06983E3
:101A60000E94B40C6981E02FF0E0EE0FFF1FE558F3
:101A7000FE4FA591B4919FB7F8948C91611103C06A
:101A80001095812301C0812B8C939FBF0F90DF9114
:101A9000CF911F910F910895FC01818D228D90E0CF
:101AA000805C9F4F821B91098F7399270895FC01D9
:101AB000918D828D981731F0828DE80FF11D858D03
:101AC00090E008958FEF9FEF0895FC01918D828D36
:101AD000981761F0828DDF01A80FB11D5D968C9182
:101AE000928D9F5F9F73928F90E008958FEF9FEF8D
:101AF000089589EE9EE0892B49F080E090E0892BE3
:101B000029F00E94E90E81110C9400000895FC0157
:101B1000848DDF01A80FB11DA35ABF4F2C91848D76
:101B200090E001968F739927848FA689B7892C93AB
:101B3000A089B1898C9180648C93938D848D981346
:101B400006C00288F389E02D80818F7D808308950F
:101B5000CF93DF93EC01888D8823C9F0EA89FB8954
:101B6000808185FD05C0A889B9898C9186FD0FC04B
:101B70000FB607FCF5CF808185FFF2CFA889B98920
:101B80008C9185FFEDCFCE010E94870DE7CFDF91CD
:101B9000CF910895CF92DF92FF920F931F93CF932F
:101BA000DF931F92CDB7DEB76C0181E0D601589666
:101BB0008C9358975B969C915B975C968C915C9705
:101BC000981307C05096ED91FC915197808185FD47
:101BD0002EC0F601038D10E00F5F1F4F0F7311270A
:101BE000F02EF601848DF81211C00FB607FCF9CF64
:101BF000D6015096ED91FC915197808185FFF1CFF0
:101C0000C60169830E94870D6981EBCF838DE80F40
:101C1000F11DE35AFF4F6083D6015B960C935B97EF
:101C20005296ED91FC915397808180620CC0D60151
:101C30005696ED91FC91579760835096ED91FC91EB
:101C4000519780818064808381E090E00F90DF91E4
:101C5000CF911F910F91FF90DF90CF900895BF9289
:101C6000CF92DF92EF92FF92CF93DF93EC016A0164
:101C70007B01B22EE889F98982E08083411581EEEB
:101C8000580761057105A1F060E079E08DE390E00F
:101C9000A70196010E94EA11215031094109510919
:101CA0005695479537952795211580E1380798F087
:101CB000E889F989108260E874E88EE190E0A70174
:101CC00096010E94EA1121503109410951095695A6
:101CD000479537952795EC85FD853083EE85FF8503
:101CE0002083188EEC89FD89B082EA89FB89808186
:101CF00080618083EA89FB89808188608083EA89AA
:101D0000FB89808180688083EA89FB8980818F7D5F
:101D10008083DF91CF91FF90EF90DF90CF90BF90C5
:101D200008951F920F920FB60F9211242F938F9345
:101D30009F93EF93FF93E0912303F091240380811D
:101D4000E0912903F0912A0382FD12C090818091D5
:101D50002C038F5F8F7320912D03821751F0E09138
:101D60002C03F0E0ED5EFC4F958F80932C0301C0B7
:101D70008081FF91EF919F918F912F910F900FBED6
:101D80000F901F9018951F920F920FB60F9211246B
:101D90002F933F934F935F936F937F938F939F9373
:101DA000AF93BF93EF93FF9383E193E00E94870D7E
:101DB000FF91EF91BF91AF919F918F917F916F9123
:101DC0005F914F913F912F910F900FBE0F901F90F9
:101DD000189583E193E00E944C0D21E0892B09F4D2
:101DE00020E0822F0895109216031092150388EEBA
:101DF00093E0A0E0B0E08093170390931803A093C2
:101E00001903B0931A038CE991E090931403809323
:101E1000130385EC90E09093200380931F0384ECE0
:101E200090E0909322038093210380EC90E09093C4
:101E300024038093230381EC90E090932603809306
:101E4000250382EC90E0909328038093270386EC8F
:101E500090E090932A038093290310922C03109210
:101E60002D0310922E0310922F030895CF92DF922C
:101E7000EF92FF920F931F93CF93DF937C016A0140
:101E8000EB0100E010E00C151D0571F06991D70120
:101E9000ED91FC910190F081E02DC7010995892B0E
:101EA00019F00F5F1F4FEFCFC801DF91CF911F9146
:101EB0000F91FF90EF90DF90CF900895611571051D
:101EC00081F0DB010D900020E9F7AD01415051098F
:101ED000461B570BDC01ED91FC910280F381E02D54
:101EE000099480E090E00895EF92FF920F931F9382
:101EF000CF93DF938C017B01C0E0D0E0F701EC0FC2
:101F0000FD1F6491662359F0F801A081B181ED9124
:101F1000FC91C8010995892B11F02196EFCFCE01D4
:101F2000DF91CF911F910F91FF90EF900895DC0109
:101F3000ED91FC91DB0114964D915C9115976D919B
:101F40007C910280F381E02D09940C945E0FDC01FA
:101F5000ED91FC910190F081E02D099468EA71E027
:101F60000C945E0F0F931F93CF93DF93EC010E94AD
:101F7000740F8C01CE010E94AE0F800F911FDF9174
:101F8000CF911F910F9108958F929F92AF92BF9220
:101F9000CF92DF92EF92FF920F931F93CF93DF9335
:101FA000CDB7DEB7A1970FB6F894DEBF0FBECDBF99
:101FB0007C01C42EE52FCB01D22E19A221E02D15D4
:101FC00010F02AE0D22E8E010F5D1F4F8D2C912C28
:101FD000A12CB12C6C2D7E2FA50194010E94EA1139
:101FE0008C2DD29E80191124015011098A3014F4CD
:101FF000805D01C0895CF8018083211531054105B0
:10200000510521F0C22EE32FCA01E4CFB801C70168
:102010000E945E0FA1960FB6F894DEBF0FBECDBF33
:10202000DF91CF911F910F91FF90EF90DF90CF90B4
:10203000BF90AF909F908F900895CF92DF92EF92D4
:10204000FF920F931F93CF93DF93EC016A017B0103
:102050002115310579F4E881F9810190F081E02DB5
:10206000642FDF91CF911F910F91FF90EF90DF9040
:10207000CF9009942A303105E9F477FF1AC06DE258
:102080000E94A70F8C0144275527BA014C195D09FE
:102090006E097F092AE0CE010E94C40F800F911FB4
:1020A000DF91CF911F910F91FF90EF90DF90CF9034
:1020B00008952AE0B701A601CE01DF91CF911F91CB
:1020C0000F91FF90EF90DF90CF900C94C40F9A0186
:1020D000AB01662757FD6095762F0C941D102115D6
:1020E000310541F4DC01ED91FC910190F081E02D8E
:1020F000642F09940C94C40F9A01462F50E060E0BD
:1021000070E00C946F100F931F93CF93DF93EC014B
:102110000E94220C688779878A879B87E881F981EA
:102120000680F781E02DCE01099597FF15C00E942A
:10213000220C088519852A853B85601B710B820B53
:10214000930B0C811D812E813F81601771078207DF
:10215000930720F38FEF9FEFDF91CF911F910F91A6
:102160000895FC0144835583668377830895CF9255
:10217000DF92EF92FF920F931F93CF93DF937C0137
:102180006A01EB0100E010E00C151D0549F0C701E4
:102190000E94831097FD04C089930F5F1F4FF4CFF7
:1021A000C801DF91CF911F910F91FF90EF90DF90C9
:1021B000CF900895FC01808191810C94F712CF9308
:1021C000DF93EC0188819981009711F00E94F7124A
:1021D000198218821D821C821B821A82DF91CF9184
:1021E00008950F931F93CF93DF93EC018B016F5FE3
:1021F0007F4F888199810E948613009731F09983DF
:1022000088831B830A8381E001C080E0DF91CF9146
:102210001F910F910895CF93DF93EC0188819981ED
:10222000892B29F08A819B818617970760F4CE015C
:102230000E94F110882341F08C819D81892B19F433
:10224000E881F981108281E0DF91CF910895EF92CA
:10225000FF920F931F93CF93DF93EC017B018A01D1
:10226000BA010E940B11811104C0CE010E94DF103F
:1022700007C01D830C83B701888199810E94AC142B
:10228000CE01DF91CF911F910F91FF90EF900895B4
:10229000FC01118210821382128215821482611550
:1022A000710559F0FB0101900020E9F7AF014150A1
:1022B0005109461B570B0C9427110895CF93DF93B8
:1022C000EC016115710561F0FB0101900020E9F757
:1022D000AF0141505109461B570B0E94271102C004
:1022E0000E94DF10CE01DF91CF910895EF92FF920F
:1022F0000F931F93CF93DF93EC017B010C811D8122
:102300006115710511F480E016C04115510591F079
:10231000040F151FB8010E940B118823A1F3288117
:1023200039818C819D81B701820F931F0E94AC146B
:102330001D830C8381E0DF91CF911F910F91FF905E
:10234000EF900895CF93DF9300D0CDB7DEB76983C8
:102350001A8241E050E0BE016F5F7F4F0E9476110C
:102360000F900F90DF91CF91089508950E94790CFE
:102370000E94B5110E940402C9E7DDE00E946606D2
:102380002097E1F30E94790DF9CF0895DB018F9337
:102390009F930E943A12BF91AF91A29F800D911D11
:1023A000A39F900DB29F900D1124089597FB072EC7
:1023B00016F4009407D077FD09D00E94451207FC5F
:1023C00005D03EF4909581959F4F08957095619545
:1023D0007F4F0895A1E21A2EAA1BBB1BFD010DC061
:1023E000AA1FBB1FEE1FFF1FA217B307E407F507C5
:1023F00020F0A21BB30BE40BF50B661F771F881FA1
:10240000991F1A9469F760957095809590959B0136
:10241000AC01BD01CF010895052E97FB1EF4009479
:102420000E94231257FD07D00E94EA1107FC03D037
:102430004EF40C94231250954095309521953F4FC2
:102440004F4F5F4F089590958095709561957F4FA0
:102450008F4F9F4F0895A29FB001B39FC001A39FCC
:10246000700D811D1124911DB29F700D811D1124CD
:10247000911D08950E942B12A59F900DB49F900D61
:10248000A49F800D911D11240895AA1BBB1B51E12F
:1024900007C0AA1FBB1FA617B70710F0A61BB70BD4
:1024A000881F991F5A95A9F780959095BC01CD0179
:1024B0000895EE0FFF1F0590F491E02D0994CF933E
:1024C000DF938230910510F482E090E0E091B20356
:1024D000F091B30320E030E0A0E0B0E0309739F1B4
:1024E0004081518148175907B8F04817590771F4CE
:1024F00082819381109729F013969C938E93129763
:102500002CC09093B3038093B20327C021153105EB
:1025100031F04217530718F0A901DB0101C0EF01A8
:102520009A01BD01DF010280F381E02DD7CF211593
:102530003105F9F0281B390B2430310580F48A81EC
:102540009B816115710521F0FB019383828304C097
:102550009093B3038093B203FE01329644C0FE0110
:10256000E20FF31F8193919322503109398328831D
:102570003AC02091B0033091B103232B41F4209154
:102580000201309103013093B1032093B0032091F5
:102590000001309101012115310541F42DB73EB7FD
:1025A0004091040150910501241B350BE091B003CB
:1025B000F091B103E217F307A0F42E1B3F0B28178D
:1025C000390778F0AC014E5F5F4F2417350748F0AC
:1025D0004E0F5F1F5093B1034093B00381939193CB
:1025E00002C0E0E0F0E0CF01DF91CF910895CF93FA
:1025F000DF93009709F487C0FC013297138212829F
:10260000C091B203D091B303209781F4208131812E
:10261000280F391F8091B0039091B103821793075F
:1026200079F5F093B103E093B0036DC0DE0120E0D3
:1026300030E0AE17BF0750F412964D915C9113979E
:102640009D014115510509F1DA01F3CFB383A2834E
:1026500040815181840F951F8A179B0771F48D91DA
:102660009C911197840F951F0296918380831296F7
:102670008D919C911397938382832115310529F4C1
:10268000F093B303E093B2033EC0D9011396FC93D9
:10269000EE9312974D915D91A40FB51FEA17FB07BA
:1026A00079F480819181840F951F0296D90111964A
:1026B0009C938E938281938113969C938E93129711
:1026C000E0E0F0E08A819B81009719F0FE01EC01C7
:1026D000F9CFCE01029628813981820F931F209174
:1026E000B0033091B1032817390769F4309729F402
:1026F0001092B3031092B20302C013821282D093DD
:10270000B103C093B003DF91CF910895A0E0B0E092
:10271000ECE8F3E10C94FB14EC01CB01209719F4E5
:102720000E945F12B8C0FE01E60FF71F9E01225003
:102730003109E217F30708F4ACC0D9010D911C91DF
:10274000119706171707B8F00530110508F49FC058
:10275000A801445051094617570708F498C0025081
:102760001109061B170B019311936D937C93CF01F5
:102770000E94F7128CC05B01A01AB10A4E01800EB4
:10278000911EA091B203B091B303612C712C60E053
:1027900070E0109709F449C0A815B905C9F5ED9086
:1027A000FC901197670142E0C40ED11CCA14DB04EF
:1027B00078F147018A189B08640142E0C40ED11CDD
:1027C0001296BC9012971396AC91B5E0CB16D1043B
:1027D00040F0B282A38391828082D9018D939C9331
:1027E00009C00E5F1F4F0E0D1F1DF90111830083DD
:1027F000EB2DFA2F6115710531F0DB011396FC9377
:10280000EE93129744C0F093B303E093B2033FC03A
:102810006D917C9111976616770608F43B01BD0116
:1028200012960D90BC91A02DB4CF6091B003709121
:10283000B10368157905E9F468167906D0F440917A
:102840000001509101014115510541F44DB75EB7AA
:102850006091040170910501461B570BE417F507C1
:10286000C0F4F093B103E093B003F9019183808346
:102870000EC00E945F127C01009759F0A801BE01B2
:102880000E949A14CE010E94F712C70104C0CE0123
:1028900002C080E090E0CDB7DEB7EEE00C941715F3
:1028A000FC0188279927E89421912032E9F3293007
:1028B00010F02E30C8F32B3241F02D3239F46894E9
:1028C00004C00E94EF14820F911D219120532A30E1
:1028D000C0F31EF4909581959F4F08951F93FC01BE
:1028E00099278827BC01E89411911032E9F3193037
:1028F00010F01E30C8F31B3251F01D3249F46894B9
:1029000006C00E94DA14610F711D811D911D119185
:1029100010531A30B0F33EF4909580957095619500
:102920007F4F8F4F9F4F1F91089548EB51E00E94BA
:10293000B3140895FB01DC0102C001900D924150D7
:102940005040D8F70895FB01DC018D91019080196A
:102950000110D9F3990B0895FB01DC0101900D9250
:102960000020E1F70895FA01A191B081009719F4D0
:102970001097E1F0CD01DC01CD010D90002011F4A4
:10298000C00113C0FB012191222319F02015D9F7B2
:10299000F3CFFB012191201519F41E92119606C068
:1029A0002223C1F70D900020A1F7D001FA01A193D5
:1029B000B0830895592F482F372F262F660F771F82
:1029C000881F991F660F771F881F991F620F731F3B
:1029D000841F951F660F771F881F991F08957AE03F
:1029E000979F902D879F802D910D112408952F92F0
:1029F0003F924F925F926F927F928F929F92AF928F
:102A0000BF92CF92DF92EF92FF920F931F93CF93DB
:102A1000DF93CDB7DEB7CA1BDB0B0FB6F894DEBF72
:102A20000FBECDBF09942A88398848885F846E8498
:102A30007D848C849B84AA84B984C884DF80EE80E2
:102A4000FD800C811B81AA81B981CE0FD11D0FB6EB
:102A5000F894DEBF0FBECDBFED01089511E0C4E9CB
:102A6000D1E004C0FE010E945B122296C639D10754
:062A7000C9F7F894FFCF46
:102A76000000B40380002C010000690B690B3A00CA
:102A86002C004A616E00466562004D61720041701D
:102A960072004D6179004A756E004A756C00417589
:102AA6006700536570004F6374004E6F760044658F
:102AB6006300244745545645520024434C4F434B2C
:102AC60000245354415455530024455854535441FB
:102AD60054555300245355525645590024474554DE
:102AE600504F53002C20002020002E000000000034
:102AF6002107360F8E070007740773071F1C1F1E5A
:102B06001F1E1F1F1E1F1E1F00000000CA0D360FAE
:102B16004C0D650D570DA80D0D0A006E616E00690E
:082B26006E66006F7666000088
:00000001FF
